:040000008A11112828
:10000800FE00030EF1000408F2000A08F300831250
:1000180003137F08F4008A11522A8A111328F80161
:100028008313373084004A308A11402383018A11B0
:100038001D288B010730831203139F0001308500B0
:1000480001308316031385008312031386010230DF
:1000580083160313860006308312031381008B1660
:1000680004308316031381007D3083120313B30019
:100078003308CA00BE01BD01F8107810B701B801F5
:10008800C001C101BF01B901F811BA01BB010030BB
:10009800A0000030A1000830A2000030A3004230C8
:1000A8008A11F6228A117811781283120313061026
:1000B8008A1119238A118B178312031385143D089B
:1000C800023A0319F81C6F2878186F288A114823F8
:1000D8008A117814F810831203133D08043A03199F
:1000E800F81C7A288A114D238A11F81083120313F9
:1000F8003D08063A0319F81C85288A1161218A11DE
:10010800F810831203138C1EA2281930B300330889
:10011800BC000430B3003308B9008C129818962834
:10012800181D9D28981C9A2818121816181DA22800
:100138009E28F8151A08B3003308BA00BC0803193A
:10014800BB01F81DB82808303B020318B828F8117D
:100158003A08B3003B08423E84003308831380000A
:100168000130B3003308BB0708303B02031CE82802
:10017800B501B601073036020318DD283608423EBD
:10018800840083130008B3003308F5003608013EE5
:100198008A112D238A11831203133507B4003408FA
:1001A800B5000130B3003308B60707303602031C28
:1001B800C22849083506031DE72842080E3A031DE0
:1001C800E7287815E828BB01781D632878114308CB
:1001D800C13A031DF428C230B3003308C4007816AE
:1001E8004308023A031D0D293708B3003308C40039
:1001F8003808B3003308C5004008B3003308C60008
:100208004108B3003308C7003F08B3003308C800EB
:100218007816781E5F297812B501B60107303602C4
:10022800031831293608423E840083130008B300BE
:100238003308F5003608013E8A112D238A118312EE
:1002480003133507B4003408B5000130B300330890
:10025800B60707303602031C16293508B3003308E1
:10026800C9000614B6010830360203185E290430A6
:10027800B3003308B9003608423E840083130008EF
:1002880099001930B3003308BC008316031398187B
:10029800522983120313BC08031D49298312BC0881
:1002A80003195E290130B3003308B6070830360257
:1002B800031C3B290610BB01632883120313051C8A
:1002C800102A8A11C3228A1183120313A700270850
:1002D800AB008A11C3228A1183120313A7002708CF
:1002E800AC008A11C3228A1183120313A7002708BE
:1002F800AD008A11C3228A1183120313A7002708AD
:10030800AE002C08A700A8012B08A900AA012908FB
:10031800AA00A90127082904B10028082A04B20064
:1003280003303202E830031931020318AD293109CC
:10033800A7003209A800A70A0319A80A2708E83E57
:10034800B10028080318013E033EB200BF01BF0AEE
:10035800B6293108183EB10032080318013EFC3EA8
:10036800B200BF010A30A0000030A1003208A3018A
:10037800A3073108A201A2078A1112228A11831247
:1003880003132008A7002708C0000A30A000003087
:10039800A1003208A301A3073108A201A2078A110C
:1003A8008D228A11831203132008A7002708C10091
:1003B8002E08A700A8012D08A900AA012908AA004B
:1003C800A90127082904AF0028082A04B0006430CE
:1003D800A0000030A1003008A301A3072F08A20144
:1003E800A2078A1112228A11831203132008A70078
:1003F8002708B7006430A0000030A1003008A3012E
:10040800A3072F08A201A2078A118D2283120313C2
:100418002008A7002708B800061208008312031353
:10042800A501A6012108200403194B2AA401A40A46
:10043800A11B2A2A01300310A00DA10DFF3E031DA8
:100448001F2A0130F5007508A4071C2A0130031083
:10045800A50DA60DFF3E031D2B2A21082302031D0F
:10046800372A20082202031C402A2008A202210859
:10047800031CA303A302251401300310A10CA00C34
:10048800FF3E031D412A0130A402031D2A2A260823
:10049800A101A1072508A001A00708000B1D822AB9
:1004A8000B11063081000130CA02CA08031D6D2AEB
:1004B8007D30F0007008CA000430F0007008BE00FB
:1004C8000130F0007008BD070A303D020318BD0175
:1004D800F8143E080319742A0130BE020515752A5E
:1004E8000511390803197C2A0130B90285157D2ABE
:1004F80085113C080319822A0130BC027408FF00E8
:1005080073088A0072088400710E8300FE0E7E0E46
:10051800090083120313210820040319BC2AF601D9
:10052800F60AA11BA32A01300310A00DA10DFF3E5E
:10053800031D982A0130F5007508F607952A210849
:100548002302031DA92A20082202031CB12A20081D
:10055800A2022108031CA303A30201300310A10C6B
:10056800A00CFF3E031DB22A0130F602031DA32A88
:100578002308A101A1072208A001A00708008312EF
:100588000313A101A001A00A093020020318F42ACC
:1005980086121830F500F50BCF2AD22A83120313DE
:1005A80086162108F5007507F6007608A100051CD7
:1005B800E02A21080138E22A2108FE39F5007508E9
:1005C800A1001830F500F50BE72AEA2A0130F500FA
:1005D800750883120313A00709302002031CCC2AD4
:1005E80021080800F6007608F5007508F7000130C4
:1005F80083120313A2020030031CA303A302FF30DB
:100608002306031D092BFF30220603190800831255
:1006180003132008F5007708840075088313800009
:100628000130F5007508F707FB2A83160313181520
:100638000C30990018128312031398171813831695
:10064800031318138312031318168316031398162B
:10065800080083120313A100A001211C372B750881
:10066800F6007608A0070310F50D0310A10CA108E9
:10067800031D312B2008080064008001840A040649
:10068800031900340406412B83120313061286163D
:0A0698000800831203130616080081
:02400E0061FF50
:00000001FF
